:1000000000308A00AA2800002630840083130008EC
:10001000031918280130F800F701F70B0D28F80B29
:100020000C284A30F700F70B13281628800B0A28F3
:1000300008000430A500C830A6000420A50B1B282A
:1000400083160610831206142408A500A50AA5032A
:1000500003192E28FF30A600042027282308A60015
:100060000420831606108312061008001230A8021E
:10007000031C4928283084008313FC3080050310BA
:10008000800C800C00080319492847280000800BC9
:100090004628080083168611831286152608A700B5
:1000A000A70AA70303195828FF30A80036205128B3
:1000B0002508A8003620831686118312861126088B
:1000C000A700A70AA70303196928FF30A800362054
:1000D00062282508A80036200800A3012308633CF5
:1000E000031C79280430A6001330A5004A20A30A77
:1000F0006E288A11CD28A4016430A3002408033C93
:10010000031C9128031D88282308E73C031C912821
:100110002408A6002308A5004A20A30A0319A40A5C
:100120007E288A11DF280330A400E830A300A40849
:10013000031D9E282308643C0318A8282408A60051
:100140002308A5004A2023080319A403A303972822
:100150008A11E02803081F398300623083168F005C
:1001600090010F0807309C008313861183128611BB
:10017000A101210BC1280130A4009030A300192057
:10018000C528A4010A30A3001920831686148312FF
:10019000861CCD280130A1006D2883160615831218
:1001A000061DE2280330A4008430A300192001308A
:1001B000A100A2012208033C031CE2287B2893280B
:0801C000A20ADA28B928630045
:04400E00103FFF3F21
:00000001FF
